:020000040000FA
:0408000063EF09F0A9
:1008100003B283EF05F0F2B4A1EF05F09EB0A9EFAB
:1008200005F09EB2B1EF05F0F2A81AEF04F0F2B2B3
:1008300032EF04F09EB61FEF04F012EF09F09E961F
:1008400000011450000A06E000011450010A06E0FD
:1008500012EF09F081EC20F012EF09F079EC22F0B0
:1008600012EF09F0CD90F2929EA03CEF04F001014E
:10087000533F3CEF04F0542BAEC1B2F1AFC1B3F122
:10088000B0C1B4F1B1C1B5F1AAC1AEF1ABC1AFF124
:10089000ACC1B0F1ADC1B1F1A6C1AAF1A7C1ABF134
:1008A000A8C1ACF1A9C1ADF1A2C1A6F1A3C1A7F144
:1008B000A4C1A8F1A5C1A9F19EC1A2F19FC1A3F154
:1008C000A0C1A4F1A1C1A5F19AC19EF19BC19FF164
:1008D0009CC1A0F19DC1A1F196C19AF197C19BF174
:1008E00098C19CF199C19DF1CECF96F1CFCF97F1F0
:1008F00053C198F154C199F1CF6ACE6A0101536B8B
:10090000546B9E90CD800FBC0F8E0FBA8BEF04F00E
:100910000F8A12EF09F00F8C0FBEC7EF04F096C1DB
:100920009AF197C19BF198C19CF199C19DF19AC12F
:100930009EF19BC19FF19CC1A0F19DC1A1F19EC1FF
:10094000A2F19FC1A3F1A0C1A4F1A1C1A5F1A2C1CF
:10095000A6F1A3C1A7F1A4C1A8F1A5C1A9F1A6C19F
:10096000AAF1A7C1ABF1A8C1ACF1A9C1ADF1AAC16F
:10097000AEF1ABC1AFF1ACC1B0F1ADC1B1F1AEC13F
:10098000B2F1AFC1B3F1B0C1B4F1B1C1B5F1010180
:100990005E6B5F6B606B616B96515E2797515F2357
:1009A00098516023995161239A515E279B515F238F
:1009B0009C5160239D5161239E515E279F515F236F
:1009C000A0516023A1516123A2515E27A3515F234F
:1009D000A4516023A5516123A6515E27A7515F232F
:1009E000A8516023A9516123AA515E27AB515F230F
:1009F000AC516023AD516123AE515E27AF515F23EF
:100A0000B0516023B1516123B2515E27B3515F23CE
:100A1000B4516023B5516123D89001016133603333
:100A20005F335E33D8900101613360335F335E33EF
:100A3000D8900101613360335F335E3300C10CF144
:100A400001C10DF102C10EF103C10FF104C110F19A
:100A500005C111F106C112F107C113F108C114F16A
:100A600009C115F10AC116F10BC117F134C135F1F5
:100A700011B846EF05F00101620E046F010E056F1B
:100A8000000E066F000E076F4FEF05F00101A70E75
:100A9000046F020E056F000E066F000E076F5EC139
:100AA00000F15FC101F160C102F161C103F118EC15
:100AB0001FF003BF04D019BE02D019A0108C11A0E2
:100AC00067EF05F010BA67EF05F00F80108A0CC1D0
:100AD00000F10DC101F10EC102F10FC103F110C10E
:100AE00004F111C105F112C106F113C107F114C1DE
:100AF00008F115C109F116C10AF117C10BF135C191
:100B000034F112EF09F00392ABB2AB98AB8803015A
:100B100003EE00F080517F0BE92604C0EFFF802B2D
:100B20008151805D700BD8A48B8200008051815D63
:100B3000700BD8A48B9281518019D8B4079012EF12
:100B400009F0F2940101453F12EF09F0462B12EF34
:100B500009F09E900101533F12EF09F0542B12EF60
:100B600009F09E9211B820EF07F08BB4BFEF05F0AB
:100B700010ACBFEF05F08B84109CC0EF05F08B9498
:100B8000C3CF55F1C4CF56F1C28207B42AEF06F0A5
:100B900047C14BF148C14CF149C14DF14AC14EF139
:100BA0005EC162F15FC163F160C164F161C165F171
:100BB00096C1B6F197C1B7F198C1B8F199C1B9F131
:100BC0009AC1BAF19BC1BBF19CC1BCF19DC1BDF101
:100BD0009EC1BEF19FC1BFF1A0C1C0F1A1C1C1F1D1
:100BE000A2C1C2F1A3C1C3F1A4C1C4F1A5C1C5F1A1
:100BF000A6C1C6F1A7C1C7F1A8C1C8F1A9C1C9F171
:100C0000AAC1CAF1ABC1CBF1ACC1CCF1ADC1CDF140
:100C1000AEC1CEF1AFC1CFF1B0C1D0F1B1C1D1F110
:100C2000B2C1D2F1B3C1D3F1B4C1D4F1B5C1D5F1E0
:100C3000010155515B2756515C23E86A5D230E2E56
:100C40002AEF06F05CC157F15DC158F15B6B5C6B3C
:100C50005D6B078E0201002F12EF09F03C0E006F52
:100C60001A50E00BE00AE866128818BE02D018B4E9
:100C7000108E00C10CF101C10DF102C10EF103C1D2
:100C80000FF104C110F105C111F106C112F107C144
:100C900013F108C114F109C115F10AC116F10BC114
:100CA00017F134C135F101018A675EEF06F08B67F9
:100CB0005EEF06F08C675EEF06F08D6762EF06F080
:100CC00092EF06F08EC100F18FC101F190C102F1E7
:100CD00091C103F10101010E046F000E056F000EBA
:100CE000066F000E076F18EC1FF000C18EF101C1F6
:100CF0008FF102C190F103C191F1006787EF06F017
:100D0000016787EF06F0026787EF06F0036792EF4F
:100D100006F08AC18EF18BC18FF18CC190F18DC12B
:100D200091F10F80D57ED5BE6DD0D6CF47F1D7CF0C
:100D300048F145C149F1E86AE8CF4AF119BE02D04D
:100D400019A0108C109047C100F148C101F149C1B0
:100D500002F14AC103F101010A0E046F000E056F92
:100D6000000E066F000E076F18EC1FF003AF108027
:100D7000010154A7C8EF06F00F9A0F9C0F9E0101C6
:100D8000000E5E6F600E5F6F3D0E606F080E616F4C
:100D9000010147BFD8EF06F04867D8EF06F0496772
:100DA000D8EF06F04A67D8EF06F0F288FDEF06F0BC
:100DB000F2985E6B5F6B606B616B966B976B986B79
:100DC000996B9A6B9B6B9C6B9D6B9E6B9F6BA06BE7
:100DD000A16BA26BA36BA46BA56BA66BA76BA86B97
:100DE000A96BAA6BAB6BAC6BAD6BAE6BAF6BB06B47
:100DF000B16BB26BB36BB46BB56BD76AD66A0101DA
:100E0000456B466B0CC100F10DC101F10EC102F141
:100E10000FC103F110C104F111C105F112C106F1B6
:100E200013C107F114C108F115C109F116C10AF186
:100E300017C10BF135C134F112EF09F012EF09F0CF
:100E40000201002F79EF08F0D59ED6CF47F1D7CF1A
:100E500048F145C149F1E86AE8CF4AF1D76AD66A54
:100E60000101456B466BD58E1A50E00BE00AE8662F
:100E7000128818BE02D018B4108E17AE1C8C00C198
:100E80000CF101C10DF102C10EF103C10FF104C15A
:100E900010F105C111F106C112F107C113F108C12A
:100EA00014F109C115F10AC116F10BC117F134C1D2
:100EB00035F10FA0109A11B869EF07F00101620E29
:100EC000046F010E056F000E066F000E076F72EFC4
:100ED00007F00101A70E046F020E056F000E066FEA
:100EE000000E076F47C100F148C101F149C102F18D
:100EF0004AC103F118EC1FF003BF85EF07F019BEDC
:100F000002D019A0108C11B00F800CC100F10DC1DE
:100F100001F10EC102F10FC103F110C104F111C1C1
:100F200005F112C106F113C107F114C108F115C191
:100F300009F116C10AF117C10BF135C134F10201F3
:100F40003C0E006F00C10CF101C10DF102C10EF1A8
:100F500003C10FF104C110F105C111F106C112F175
:100F600007C113F108C114F109C115F10AC116F145
:100F70000BC117F134C135F101018A67C7EF07F0E2
:100F80008B67C7EF07F08C67C7EF07F08D67CBEF74
:100F900007F0FBEF07F08EC100F18FC101F190C1A6
:100FA00002F191C103F10101010E046F000E056F02
:100FB000000E066F000E076F18EC1FF000C18EF1D7
:100FC00001C18FF102C190F103C191F10067F0EF0F
:100FD00007F00167F0EF07F00267F0EF07F0036733
:100FE000FBEF07F08AC18EF18BC18FF18CC190F1BC
:100FF0008DC191F10F80109047C100F148C101F1FE
:1010000049C102F14AC103F101010A0E046F000E49
:10101000056F000E066F000E076F18EC1FF003AF90
:101020001080010154A721EF08F00F9A0F9C0F9E2A
:101030000101000E5E6F600E5F6F3D0E606F080E67
:10104000616F47C100F148C101F149C102F14AC1D4
:1010500003F10101140E046F050E056F000E066FFB
:10106000000E076F18EC1FF003AF3AEF08F0F2889C
:101070005FEF08F0F2985E6B5F6B606B616B966B75
:10108000976B986B996B9A6B9B6B9C6B9D6B9E6B34
:101090009F6BA06BA16BA26BA36BA46BA56BA66BE4
:1010A000A76BA86BA96BAA6BAB6BAC6BAD6BAE6B94
:1010B000AF6BB06BB16BB26BB36BB46BB56B0CC198
:1010C00000F10DC101F10EC102F10FC103F110C118
:1010D00004F111C105F112C106F113C107F114C1E8
:1010E00008F115C109F116C10AF117C10BF135C19B
:1010F00034F138EC23F01D661ED01CAE11D01C9EBE
:101100001D8E18AE07D0146A040E156E166A81EC97
:1011100020F011D0146A156A166A81EC20F00BD009
:101120001CAC09D01C9C1D8C010E146E156A166A2D
:1011300079EC22F000D08BB4A5EF08F010ACA5EF4D
:1011400008F08B84109CA6EF08F08B94C3CF55F168
:10115000C4CF56F1C28207B410EF09F047C14BF17A
:1011600048C14CF149C14DF14AC14EF15EC162F135
:101170005FC163F160C164F161C165F196C1B6F10F
:1011800097C1B7F198C1B8F199C1B9F19AC1BAF153
:101190009BC1BBF19CC1BCF19DC1BDF19EC1BEF123
:1011A0009FC1BFF1A0C1C0F1A1C1C1F1A2C1C2F1F3
:1011B000A3C1C3F1A4C1C4F1A5C1C5F1A6C1C6F1C3
:1011C000A7C1C7F1A8C1C8F1A9C1C9F1AAC1CAF193
:1011D000ABC1CBF1ACC1CCF1ADC1CDF1AEC1CEF163
:1011E000AFC1CFF1B0C1D0F1B1C1D1F1B2C1D2F133
:1011F000B3C1D3F1B4C1D4F1B5C1D5F10101555199
:101200005B2756515C23E86A5D230E2E10EF09F030
:101210005CC157F15DC158F15B6B5C6B5D6B078E18
:1012200012EF09F002C0E0FF005001C0D8FF10002B
:10123000A6B218EF09F00CC0A9FF0BC0A8FFA69E2C
:10124000A69CA684F29E550EA76EAA0EA76EA68235
:10125000F28EA694A6B22AEF09F00C2A1200A96E0B
:10126000A69EA69CA680A8500C2A120004012C0E53
:10127000826F3BEC0BF013EC20F00C502FEC09F0DC
:10128000E8CF00F10C502FEC09F0E8CF01F101AFED
:101290004FEF09F00101FF0E026FFF0E036FB6EC76
:1012A0001FF029675BEF09F00401200E826F3BEC11
:1012B0000BF060EF09F004012D0E826F3BEC0BF098
:1012C000C0EC1DF01200306A076A0F6A106A116ADA
:1012D000126A136A0F010E0EC16E860EC06E030EE7
:1012E000C26E0F01896A110E926E080E8A6EF10E9F
:1012F000936E8B6A980E946EF18EFC0E2FEC09F0B3
:10130000E8CF0BF00BA011800BA211820BA411846B
:101310000BA81188C90E2FEC09F0E8CF17F0CA0E00
:101320002FEC09F0E8CF18F0CB0E2FEC09F0E8CF46
:1013300019F0CC0E2FEC09F0E8CF1AF0CD0E2FECFF
:1013400009F0E8CF2FF01C6A1D6A0E6A01015B6B81
:101350005C6B5D6B576B586BF29A0101476B486B86
:10136000496B4A6B4B6B4C6B4D6B4E6B4F6B506BC1
:10137000516B526B456B466BD76AD66A0F01280ECC
:10138000D56EF28A9D90B00ECD6E01015E6B5F6BE3
:10139000606B616B626B636B646B656B666B676BD9
:1013A000686B696B536B546BCF6ACE6A0F9A0F9C54
:1013B0000F9E9D80760ECA6E9D8202013C0E006FCC
:1013C000CC6A160E2FEC09F0E8CF00F1170E2FECC7
:1013D00009F0E8CF01F1180E2FEC09F0E8CF02F187
:1013E000190E2FEC09F0E8CF03F1010103AF13EF61
:1013F0000AF013EC20F0160E0C6E00C10BF018EC86
:1014000009F0170E0C6E01C10BF018EC09F0180E64
:101410000C6E02C10BF018EC09F0190E0C6E03C132
:101420000BF018EC09F000C18AF101C18BF102C187
:101430008CF103C18DF100C18EF101C18FF102C1A8
:1014400090F103C191F11A0E2FEC09F0E8CF00F1F1
:101450001B0E2FEC09F0E8CF01F11C0E2FEC09F068
:10146000E8CF02F11D0E2FEC09F0E8CF03F10101E6
:1014700003AF69EF0AF013EC20F01A0E0C6E00C1F6
:101480000BF018EC09F01B0E0C6E01C10BF018EC00
:1014900009F01C0E0C6E02C10BF018EC09F01D0EC9
:1014A0000C6E03C10BF018EC09F01A0E2FEC09F0CA
:1014B000E8CF00F11B0E2FEC09F0E8CF01F11C0E74
:1014C0002FEC09F0E8CF02F11D0E2FEC09F0E8CF68
:1014D00003F100C192F101C193F102C194F103C182
:1014E00095F1240EAC6E900EAB6E240EAC6E080E11
:1014F000B86E000EB06E1F0EAF6E0401806B816B74
:101500000F01900EAB6E0F019D8A0301806B816B02
:10151000C26B8B92146A156A166A9D860790000149
:10152000F28EF28C07B069EF1CF00FB0FDEF15F0F2
:1015300010BEFDEF15F012B8FDEF15F0030180515C
:1015400081197F0BD8B469EF1CF013EE00F08151C4
:101550007F0BE126812BE7CFE8FFE00BD8B469EFE2
:101560001CF023EE82F0C2513F0BD926E7CFDFFFFC
:10157000C22BDF50780AD8A469EF1CF007808EC117
:1015800000F18FC101F190C102F191C103F101019C
:10159000040E046F000E056F000E066F000E076F3D
:1015A00018EC1FF000AFDEEF0AF00101030E8E6FA2
:1015B000000E8F6F000E906F000E916F030182512D
:1015C000720AD8B4E1EF15F08251520AD8B4E1EFB3
:1015D00015F08251750AD8B4E1EF15F08251630A13
:1015E000D8B423EF19F08251690AD8B488EF12F009
:1015F00082517A0AD8B49BEF13F08251490AD8B4C9
:1016000027EF12F08251500AD8B431EF11F0825115
:10161000700AD8B479EF11F08251540AD8B4A9EF06
:1016200011F08251740AD8B4F4EF11F08251410ADA
:10163000D8B451EF0CF082514B0AD8B44FEF0BF0F5
:1016400082516D0AD8B484EF10F082514D0AD8B49B
:101650009DEF10F08251730AD8B411EF15F082514A
:10166000530AD8B476EF15F08251590AD8B4D5EFA1
:101670000FF05AEF19F0040114EE00F080517F0BC7
:10168000E12682C4E7FF802B120004010D0E826F59
:101690003BEC0BF00A0E826F3BEC0BF012000401E6
:1016A0004B0E826F3BEC0BF004012C0E826F3BEC77
:1016B0000BF081B802D02FB630D003018351430A1A
:1016C000D8B494EF0BF003018351630AD8B496EFBA
:1016D0000BF003018351520AD8B498EF0BF00301C9
:1016E0008351720AD8B49AEF0BF003018351470A71
:1016F000D8B49CEF0BF003018351670AD8B49EEF76
:101700000BF003018351540AD8B4A0EF0BF003018E
:101710008351740AD8B40FEF0CF003018351550ABA
:10172000D8B4A2EF0BF082D02F807AD02F9078D04F
:101730002F8276D02F9274D02F8472D02F9470D0B5
:101740002F866ED084C330F185C331F186C332F168
:1017500087C333F10101296B61EC20F0D8EC1FF055
:1017600000C104F101C105F102C106F103C107F195
:1017700054EC20F0200EF86EF76AF66A0900F5CFF7
:101780002CF10900F5CF2DF10900F5CF2EF109005C
:10179000F5CF2FF10900F5CF30F10900F5CF31F188
:1017A0000900F5CF32F10900F5CF33F10101296BC2
:1017B00061EC20F0D8EC1FF018EC1FF00067E8EFA8
:1017C0000BF00167E8EF0BF00267E8EF0BF003673F
:1017D00001D025D004014E0E826F3BEC0BF00401CA
:1017E0006F0E826F3BEC0BF004014D0E826F3BECF1
:1017F0000BF00401610E826F3BEC0BF00401740EE0
:10180000826F3BEC0BF00401630E826F3BEC0BF03C
:101810000401680E826F3BEC0BF058EF19F02F9625
:10182000CD0E0C6E2FC00BF018EC09F0CD0E2FEC86
:1018300009F0E8CF2FF02FB006D00401630E826FBD
:101840003BEC0BF005D00401430E826F3BEC0BF038
:101850002FB206D00401720E826F3BEC0BF005D064
:101860000401520E826F3BEC0BF02FB406D0040142
:10187000670E826F3BEC0BF005D00401470E826FC0
:101880003BEC0BF02FB606D00401740E826F3BECDC
:101890000BF005D00401540E826F3BEC0BF058EFB7
:1018A00019F00401410E826F3BEC0BF003018351F0
:1018B000310AD8B4F5EF0EF003018351320AD8B4DF
:1018C00025EF0EF003018351330AD8B4AEEF0DF0CB
:1018D00003018351340AD8B49EEF0CF00301835105
:1018E000350AD8B47BEF0CF004013F0E826F3BEC5D
:1018F0000BF058EF19F004012C0E826F3BEC0BF04B
:1019000003018451300AD8B48EEF0CF003018451E6
:10191000310AD8B496EF0CF0E7EF0DF08B9004018C
:10192000300E826F3BEC0BF09CEF0CF08B800401CF
:10193000310E826F3BEC0BF058EF19F0CC0E2FEC10
:1019400009F0E8CF0BF004012C0E826F3BEC0BF09A
:1019500003018451310AD8B4C2EF0CF00301845161
:10196000300AD8B4C4EF0CF0030184514D0AD8B446
:10197000CEEF0CF003018451540AD8B4D5EF0CF02B
:10198000ECEF0CF08A8401D08A940BAE04D00BAC3F
:1019900002D00BBA21D0E00E0B1218D01F0E0B167E
:1019A0008539E844E00B0B1211D0E00E0B1654EC15
:1019B00020F085C332F186C333F10101296B61EC5C
:1019C00020F0D8EC1FF000511F0B0B12CC0E0C6E48
:1019D0000BC00BF018EC09F00401340E826F3BECE5
:1019E0000BF004012C0E826F3BEC0BF0CC0E2FECB5
:1019F00009F0E8CF1AF08AB406D00401300E826FE5
:101A00003BEC0BF005D00401310E826F3BEC0BF088
:101A100004012C0E826F3BEC0BF01A38E840070BE8
:101A2000E8CF82F40401300E82273BEC0BF0040176
:101A30002C0E826F3BEC0BF013EC20F01A501F0BB6
:101A4000E8CF00F1B6EC1FF032C182F40401300E91
:101A500082273BEC0BF033C182F40401300E822765
:101A60003BEC0BF004012C0E826F3BEC0BF013EC03
:101A700020F02DC000F100AF0BD0FF0E016FFF0E64
:101A8000026FFF0E036F04012D0E826F3BEC0BF013
:101A9000B6EC1FF031C182F40401300E82273BEC1A
:101AA0000BF032C182F40401300E82273BEC0BF0C4
:101AB00033C182F40401300E82273BEC0BF00401A9
:101AC0002C0E826F3BEC0BF013EC20F02CC000F1DD
:101AD000B6EC1FF031C182F40401300E82273BECDA
:101AE0000BF032C182F40401300E82273BEC0BF084
:101AF00033C182F40401300E82273BEC0BF0040169
:101B00002C0E826F3BEC0BF013EC20F02EC000F19A
:101B100000AF0BD0FF0E016FFF0E026FFF0E036FC1
:101B200004012D0E826F3BEC0BF0B6EC1FF031C1BF
:101B300082F40401300E82273BEC0BF032C182F4B8
:101B40000401300E82273BEC0BF033C182F4040118
:101B5000300E82273BEC0BF058EF19F0CB0E2FEC38
:101B600009F0E8CF0BF004012C0E826F3BEC0BF078
:101B700003018451450AD8B4D2EF0DF0030184511A
:101B8000440AD8B4D5EF0DF003018451300AD8B41B
:101B9000D8EF0DF003018451310AD8B4DCEF0DF019
:101BA000E7EF0DF00B9EE1EF0DF00B8EE1EF0DF086
:101BB000FC0E0B16E1EF0DF0FC0E0B160B80E1EFA7
:101BC0000DF0CB0E0C6E0BC00BF018EC09F00401FD
:101BD000330E826F3BEC0BF004012C0E826F3BEC5A
:101BE0000BF0CB0E2FEC09F0E8CF19F019BE00EF87
:101BF0000EF00401450E826F3BEC0BF005EF0EF08A
:101C00000401440E826F3BEC0BF004012C0E826F3A
:101C10003BEC0BF00401300E826F3BEC0BF0040147
:101C20002C0E826F3BEC0BF019B01EEF0EF004018E
:101C3000300E826F3BEC0BF023EF0EF00401310EFF
:101C4000826F3BEC0BF058EF19F0CA0E2FEC09F045
:101C5000E8CF0BF004012C0E826F3BEC0BF003017C
:101C60008451450AD8B461EF0EF003018451440A4F
:101C7000D8B464EF0EF0030184514D0AD8B46DEF6F
:101C80000EF003018451410AD8B467EF0EF003014E
:101C90008451460AD8B46AEF0EF003018451560A03
:101CA000D8B475EF0EF003018451500AD8B480EF18
:101CB0000EF003018451520AD8B483EF0EF08CEF7A
:101CC0000EF00B9E86EF0EF00B8E86EF0EF00B9C47
:101CD00086EF0EF00B8C86EF0EF0FC0E0B1685C314
:101CE000E8FF030B0B1286EF0EF0C70E0B1685C331
:101CF000E8FF070BE846E846E8460B1286EF0EF0D1
:101D00000B8486EF0EF00B9486EF0EF0CA0E0C6E6D
:101D10000BC00BF018EC09F0CA0E2FEC09F0E8CF5D
:101D200018F00401320E826F3BEC0BF004012C0E14
:101D3000826F3BEC0BF018BEA5EF0EF00401450ED0
:101D4000826F3BEC0BF0AAEF0EF00401440E826FA1
:101D50003BEC0BF004012C0E826F3BEC0BF018C037
:101D6000E8FF030BE8CF82F40401300E82273BEC3E
:101D70000BF004012C0E826F3BEC0BF018BCC8EF8B
:101D80000EF00401410E826F3BEC0BF0CDEF0EF034
:101D90000401460E826F3BEC0BF004012C0E826FA7
:101DA0003BEC0BF018C0E8FF380BE842E842E84291
:101DB000E8CF82F40401300E82273BEC0BF00401E3
:101DC0002C0E826F3BEC0BF018B4EEEF0EF004011A
:101DD000520E826F3BEC0BF0F3EF0EF00401500E4D
:101DE000826F3BEC0BF058EF19F0C90E2FEC09F0A5
:101DF000E8CF0BF004012C0E826F3BEC0BF00301DB
:101E00008451450AD8B413EF0FF003018451440AFA
:101E1000D8B416EF0FF0030184514D0AD8B419EF6E
:101E20000FF027EF0FF00B9E21EF0FF00B8E21EF3D
:101E30000FF0F80E0B1685C3E8FF070B0B1221EF0E
:101E40000FF0C90E0C6E0BC00BF018EC09F004017A
:101E5000310E826F3BEC0BF004012C0E826F3BECD9
:101E60000BF0C90E2FEC09F0E8CF17F017BE06D023
:101E70000401450E826F3BEC0BF005D00401440ECB
:101E8000826F3BEC0BF004012C0E826F3BEC0BF0ED
:101E900017C0E8FF070BE8CF82F40401300E822759
:101EA0003BEC0BF004012C0E826F3BEC0BF0078037
:101EB00013EC20F028C0E8FF003B00430043030B75
:101EC000B6EC1FF033C182F40401300E82273BECE4
:101ED0000BF004012C0E826F3BEC0BF013EC20F0A6
:101EE00028C001F1019F019D29C000F10101B6EC5C
:101EF0001FF02FC182F40401300E82273BEC0BF05F
:101F000030C182F40401300E82273BEC0BF031C16A
:101F100082F40401300E82273BEC0BF032C182F4D4
:101F20000401300E82273BEC0BF033C182F4040134
:101F3000300E82273BEC0BF004012C0E826F3BEC41
:101F40000BF013EC20F02AC001F12BC000F1D89067
:101F500001330033D890013300330101B6EC1FF098
:101F60002FC182F40401300E82273BEC0BF030C10C
:101F700082F40401300E82273BEC0BF031C182F475
:101F80000401300E82273BEC0BF032C182F40401D5
:101F9000300E82273BEC0BF033C182F40401300E8B
:101FA00082273BEC0BF058EF19F0FC0E2FEC09F0F8
:101FB000E8CF0BF003018351520AD8B40CEF10F0B4
:101FC00003018351720AD8B40FEF10F0030183515B
:101FD000500AD8B412EF10F003018351700AD8B43C
:101FE00015EF10F003018351550AD8B418EF10F023
:101FF00003018351750AD8B41BEF10F0030183511C
:10200000430AD8B424EF10F003018351630AD8B413
:1020100027EF10F030EF10F00B902AEF10F00B804C
:102020002AEF10F00B922AEF10F00B822AEF10F03B
:102030000B942AEF10F00B842AEF10F00B962AEF86
:1020400010F00B862AEF10F00B982AEF10F00B8897
:102050002AEF10F0FC0E0C6E0BC00BF018EC09F020
:102060000401590E826F3BEC0BF011901192119408
:102070001198FC0E2FEC09F0E8CF0BF00BA01180AB
:102080000BA211820BA411840BA8118811A050EF90
:1020900010F00401520E826F3BEC0BF055EF10F084
:1020A0000401720E826F3BEC0BF011A85FEF10F091
:1020B0000401430E826F3BEC0BF064EF10F004015F
:1020C000630E826F3BEC0BF011A26EEF10F0040177
:1020D000500E826F3BEC0BF073EF10F00401700EAA
:1020E000826F3BEC0BF011A47DEF10F00401550E54
:1020F000826F3BEC0BF082EF10F00401750E826FE3
:102100003BEC0BF058EF19F004016D0E826F3BECC5
:102110000BF003018351300AD8B4E1EF10F0030152
:102120008351310AD8B4F4EF10F003018351320A1D
:10213000D8B407EF11F05AEF19F081B803D02FB4DB
:1021400058EF19F004014D0E826F3BEC0BF054EC8C
:1021500020F084C331F185C332F186C333F101012C
:10216000296B61EC20F0D8EC1FF003018351300A99
:10217000D8B4C9EF10F003018351310AD8B4D1EFBC
:1021800010F003018351320AD8B4D9EF10F05AEF9E
:1021900019F0FD0E0C6E00C10BF018EC09F0E1EF28
:1021A00010F0FE0E0C6E00C10BF018EC09F0F4EF0D
:1021B00010F0FF0E0C6E00C10BF018EC09F007EFE9
:1021C00011F00401300E826F3BEC0BF004012C0E79
:1021D000826F3BEC0BF013EC20F0FD0E2FEC09F0BE
:1021E000E8CF00F118EF11F00401310E826F3BECE3
:1021F0000BF004012C0E826F3BEC0BF013EC20F083
:10220000FE0E2FEC09F0E8CF00F118EF11F00401F9
:10221000320E826F3BEC0BF013EC20F004012C0E1D
:10222000826F3BEC0BF0FF0E2FEC09F0E8CF00F1D2
:10223000B6EC1FF031C182F40401300E82273BEC72
:102240000BF032C182F40401300E82273BEC0BF01C
:1022500033C182F40401300E82273BEC0BF058EFBF
:1022600019F081B803D02FB227EF12F083C32AF1FF
:1022700084C32BF185C32CF186C32DF187C32EF1C6
:1022800088C32FF189C330F18AC331F18BC332F196
:102290008CC333F1010161EC20F0D8EC1FF0160E75
:1022A0000C6E00C10BF018EC09F0170E0C6E01C19A
:1022B0000BF018EC09F0180E0C6E02C10BF018ECC4
:1022C00009F0190E0C6E03C10BF018EC09F000C1F7
:1022D0008AF101C18BF102C18CF103C18DF100C102
:1022E0008EF101C18FF102C190F103C191F127EF8D
:1022F00012F081B803D02FB227EF12F083C32AF176
:1023000084C32BF185C32CF186C32DF187C32EF135
:1023100088C32FF189C330F18AC331F18BC332F105
:102320008CC333F1010161EC20F0D8EC1FF000C147
:102330008AF101C18BF102C18CF103C18DF100C1A1
:102340008EF101C18FF102C190F103C191F127EF2C
:1023500012F081B803D02FB227EF12F083C32AF115
:1023600084C32BF185C32CF186C32DF187C32EF1D5
:1023700088C32FF189C330F18AC331F18CC332F1A4
:102380008DC333F1010161EC20F0D8EC1FF00101A5
:10239000000E046F000E056F010E066F000E076F32
:1023A00029EC1FF01A0E0C6E00C10BF018EC09F0AE
:1023B0001B0E0C6E01C10BF018EC09F01C0E0C6E1C
:1023C00002C10BF018EC09F01D0E0C6E03C10BF0EE
:1023D00018EC09F000C192F101C193F102C194F12E
:1023E00003C195F127EF12F081B803D02FB227EF88
:1023F00012F083C32AF184C32BF185C32CF186C369
:102400002DF187C32EF188C32FF189C330F18AC320
:1024100031F18CC332F18DC333F1010161EC20F055
:10242000D8EC1FF00101000E046F000E056F010EC5
:10243000066F000E076F29EC1FF000C192F101C179
:1024400093F102C194F103C195F127EF12F0160E3A
:102450002FEC09F0E8CF00F1170E2FEC09F0E8CFD0
:1024600001F1180E2FEC09F0E8CF02F1190E2FEC54
:1024700009F0E8CF03F1B6EC1FF079EC1DF0040190
:10248000730E826F3BEC0BF004012C0E826F3BEC61
:102490000BF08AC100F18BC101F18CC102F18DC139
:1024A00003F1B6EC1FF079EC1DF00401730E826F9E
:1024B0003BEC0BF004012C0E826F3BEC0BF01A0E80
:1024C0002FEC09F0E8CF00F11B0E2FEC09F0E8CF5C
:1024D00001F11C0E2FEC09F0E8CF02F11D0E2FECDC
:1024E00009F0E8CF03F175EC19F004012C0E826FAE
:1024F0003BEC0BF092C100F193C101F194C102F1E8
:1025000095C103F175EC19F045EC0BF05AEF19F099
:102510000401690E826F3BEC0BF004012C0E826FFC
:102520003BEC0BF00101040E006F000E016F000E7A
:10253000026F000E036FB6EC1FF02CC182F4040191
:10254000300E82273BEC0BF02DC182F40401300EDB
:1025500082273BEC0BF02EC182F40401300E82275F
:102560003BEC0BF02FC182F40401300E82273BECD0
:102570000BF030C182F40401300E82273BEC0BF0EB
:1025800031C182F40401300E82273BEC0BF032C1E2
:1025900082F40401300E82273BEC0BF033C182F44D
:1025A0000401300E82273BEC0BF004012C0E826FED
:1025B0003BEC0BF00101030E006F000E016F000EEB
:1025C000026F000E036FB6EC1FF02CC182F4040101
:1025D000300E82273BEC0BF02DC182F40401300E4B
:1025E00082273BEC0BF02EC182F40401300E8227CF
:1025F0003BEC0BF02FC182F40401300E82273BEC40
:102600000BF030C182F40401300E82273BEC0BF05A
:1026100031C182F40401300E82273BEC0BF032C151
:1026200082F40401300E82273BEC0BF033C182F4BC
:102630000401300E82273BEC0BF004012C0E826F5C
:102640003BEC0BF00101380E006F000E016F000E25
:10265000026F000E036FB6EC1FF02CC182F4040170
:10266000300E82273BEC0BF02DC182F40401300EBA
:1026700082273BEC0BF02EC182F40401300E82273E
:102680003BEC0BF02FC182F40401300E82273BECAF
:102690000BF030C182F40401300E82273BEC0BF0CA
:1026A00031C182F40401300E82273BEC0BF032C1C1
:1026B00082F40401300E82273BEC0BF033C182F42C
:1026C0000401300E82273BEC0BF004012C0E826FCC
:1026D0003BEC0BF0200EF86EF76AF66A0401090075
:1026E000F5CF82F43BEC0BF00900F5CF82F43BEC24
:1026F0000BF00900F5CF82F43BEC0BF00900F5CFAD
:1027000082F43BEC0BF00900F5CF82F43BEC0BF0CC
:102710000900F5CF82F43BEC0BF00900F5CF82F411
:102720003BEC0BF00900F5CF82F43BEC0BF045ECF1
:102730000BF05AEF19F081B803D02FB0EBEF13F084
:102740008351630AD8A458EF19F08451610AD8A4C0
:1027500058EF19F085516C0AD8A458EF19F086513A
:10276000410A42E08651440A1BE08651420AD8B42D
:1027700007EF14F08651350AD8B4E4EF1AF0865109
:10278000360AD8B439EF1BF08651370AD8B4A2EF15
:102790001BF08651380AD8B400EF1CF058EF19F03E
:1027A0000798079A04017A0E826F3BEC0BF0040144
:1027B000780E826F3BEC0BF00401640E826F3BECF1
:1027C0000BF081A8EBEF13F00401550E826F3BEC88
:1027D0000BF0F0EF13F004014C0E826F3BEC0BF0AA
:1027E00045EC0BF05AEF19F00788079A04017A0EAE
:1027F000826F3BEC0BF00401410E826F3BEC0BF05F
:102800000401610E826F3BEC0BF0E1EF13F00798CF
:10281000078A04017A0E826F3BEC0BF00401420E32
:10282000826F3BEC0BF00401610E826F3BEC0BF00E
:10283000E1EF13F00101666725EF14F0676725EFFC
:1028400014F0686725EF14F0696715D04F6730EF13
:1028500014F0506730EF14F0516730EF14F0526706
:102860000AD00101000E006F000E016F000E026F12
:10287000000E036F120011B80AD00101620E046F3E
:10288000010E056F000E066F000E076F09D00101E3
:10289000A70E046F020E056F000E066F000E076F85
:1028A00066C100F167C101F168C102F169C103F1BC
:1028B00018EC1FF003BFCDEF14F0119A119C010129
:1028C000000E046FA80E056F550E066F020E076FFF
:1028D00066C100F167C101F168C102F169C103F18C
:1028E00066C186F167C187F168C188F169C189F164
:1028F00018EC1FF003BF0BD00101000E866FA80E6D
:10290000876F550E886F020E896F118A119C0E0E0B
:102910002FEC09F0E8CF18F10F0E2FEC09F0E8CFFB
:1029200019F1100E2FEC09F0E8CF1AF1110E2FEC6F
:1029300009F0E8CF1BF161EC1EF086C104F187C1FC
:1029400005F188C106F189C107F118EC1FF0078273
:1029500025EC1EF061EC1EF0079225EC1EF086C1FE
:1029600000F187C101F188C102F189C103F1079229
:1029700025EC1EF0CC0E046FE00E056F870E066F7F
:10298000050E076F18EC1FF000C118F101C119F115
:1029900002C11AF103C11BF13BD0119C119A010134
:1029A000800E006F1A0E016F060E026F000E036F8D
:1029B0004FC104F150C105F151C106F152C107F1F7
:1029C00018EC1FF003AF05D013EC20F0118C119A16
:1029D00012000E0E2FEC09F0E8CF18F10F0E2FECBD
:1029E00009F0E8CF19F1100E2FEC09F0E8CF1AF139
:1029F000110E2FEC09F0E8CF1BF14FC100F150C1CF
:102A000001F151C102F152C103F1078225EC1EF020
:102A100018C100F119C101F11AC102F11BC103F182
:102A200012000401730E826F3BEC0BF004012C0EBC
:102A3000826F3BEC0BF0078462C166F163C167F102
:102A400064C168F165C169F14BC14FF14CC150F1EE
:102A50004DC151F14EC152F157C159F158C15AF10E
:102A6000079437EC15F045EC0BF05AEF19F066C1FE
:102A700000F167C101F168C102F169C103F101010F
:102A8000B6EC1FF079EC1DF00401630E826F3BEC95
:102A90000BF004012C0E826F3BEC0BF04FC100F1E8
:102AA00050C101F151C102F152C103F10101B6EC73
:102AB0001FF079EC1DF00401660E826F3BEC0BF009
:102AC00004012C0E826F3BEC0BF013EC20F059C18B
:102AD00000F15AC101F10101B6EC1FF079EC1DF0D3
:102AE0000401740E826F3BEC0BF0120010820401A3
:102AF000530E826F3BEC0BF004012C0E826F3BEC0B
:102B00000BF083C32AF184C32BF185C32CF186C358
:102B10002DF187C32EF188C32FF189C330F18AC309
:102B200031F18BC332F18CC333F1010161EC20F040
:102B3000D8EC1FF000C166F101C167F102C168F174
:102B400003C169F18EC32AF18FC32BF190C32CF11D
:102B500091C32DF192C32EF193C32FF194C330F1A1
:102B600095C331F196C332F197C333F1010161ECA2
:102B700020F0D8EC1FF000C14FF101C150F102C1AB
:102B800051F103C152F154EC20F099C32FF19AC3D3
:102B900030F19BC331F19CC332F19DC333F101018C
:102BA00061EC20F0D8EC1FF000C159F101C15AF1DD
:102BB00037EC15F004012C0E826F3BEC0BF0F1EFBB
:102BC00015F0118E19A002D019AE108C18BE02D0CB
:102BD00018A4108E03018251520A02E10F8201D023
:102BE0000F928251750A02E1108401D01094825133
:102BF000550A02E1108601D0109611A003D011A44D
:102C000001D01084078410B25FEF16F010A44BEFD0
:102C100016F0B6C166F1B7C167F1B8C168F1B9C1C4
:102C200069F1BAC16AF1BBC16BF1BCC16CF1BDC144
:102C30006DF1BEC16EF1BFC16FF1C0C170F1C1C114
:102C400071F1C2C172F1C3C173F1C4C174F1C5C1E4
:102C500075F1C6C176F1C7C177F1C8C178F1C9C1B4
:102C600079F1CAC17AF1CBC17BF1CCC17CF1CDC184
:102C70007DF1CEC17EF1CFC17FF1D0C180F1D1C154
:102C800081F1D2C182F1D3C183F1D4C184F1D5C124
:102C900085F153EF16F062C166F163C167F164C15B
:102CA00068F165C169F14BC14FF14CC150F14DC1A3
:102CB00051F14EC152F157C159F158C15AF107941F
:102CC0000FA081EF16F0010192676EEF16F0936787
:102CD0006EEF16F094676EEF16F0956772EF16F0D0
:102CE00081EF16F01AEC14F092C104F193C105F1D2
:102CF00094C106F195C107F118EC1FF003BF1EEF58
:102D000019F01AEC14F00101000E046F000E056FAB
:102D1000010E066F000E076F49EC1FF011A02AD0BC
:102D200011A228D0B6EC1FF0296701D005D004010C
:102D30002D0E826F3BEC0BF030C182F40401300E9B
:102D400082273BEC0BF031C182F40401300E822764
:102D50003BEC0BF032C182F40401300E82273BECD5
:102D60000BF033C182F40401300E82273BEC0BF0F0
:102D700045EC0BF012A8C5D012981AC01BF01B3AF4
:102D80001B42070E1B1600011B50000AD8B44DEF62
:102D900017F000011B50010AD8B4D9EF16F000015A
:102DA0001B50020AD8B4D7EF16F07FEF17F07FEF71
:102DB00017F013EC20F02AC001F12BC000F1D890DD
:102DC00001330033D890013300330101630E046FE7
:102DD000000E056F000E066F000E076F49EC1FF026
:102DE000280E046F000E056F000E066F000E076FB1
:102DF00018EC1FF000C12DF013EC20F028C001F1F9
:102E0000019F019D29C000F10101A40E046F000E75
:102E1000056F000E066F000E076F49EC1FF000C132
:102E20002CF000C104F101C105F102C106F103C19A
:102E300007F1640E006F000E016F000E026F000EAE
:102E4000036F18EC1FF0050E046F000E056F000EE7
:102E5000066F000E076F49EC1FF000C104F101C1BD
:102E600005F102C106F103C107F113EC20F02DC0FA
:102E700000F118EC1FF000C12EF02EC0E8FF050F86
:102E80002D5C03E78A847FEF17F02EC0E8FF0A0F5E
:102E90002D5C01E68A947FEF17F000C124F101C197
:102EA00025F102C126F103C127F113EC20F019EC42
:102EB00020F01A501F0BE8CF00F10101640E046FDF
:102EC000000E056F000E066F000E076F29EC1FF055
:102ED00024C104F125C105F126C106F127C107F17E
:102EE00018EC1FF003BF02D08A9401D08A8424C159
:102EF00000F125C101F126C102F127C103F15AEF0A
:102F000019F000C124F101C125F102C126F103C16C
:102F100027F110AE4DD0109E00C108F101C109F19A
:102F200002C10AF103C10BF1B6EC1FF030C1D6F1BA
:102F300031C1D7F132C1D8F133C1D9F108C100F1A3
:102F400009C101F10AC102F10BC103F101016C0ECB
:102F5000046F070E056F000E066F000E076F18EC6A
:102F60001FF003BF04D00101550EDA6F1CD008C159
:102F700000F109C101F10AC102F10BC103F1010124
:102F8000A40E046F060E056F000E066F000E076F8D
:102F900018EC1FF003BF04D001017F0EDA6F03D0DD
:102FA0000101FF0EDA6F1C8E11AE1EEF19F0119E9B
:102FB00024C100F125C101F126C102F127C103F1AD
:102FC00011A005D011A203D00FB01EEF19F010A46C
:102FD000F1EF17F00401750E826F3BEC0BF0F6EF8A
:102FE00017F00401720E826F3BEC0BF004012C0E03
:102FF000826F3BEC0BF0B6EC1FF0296705EF18F081
:103000000401200E826F08EF18F004012D0E826F6C
:103010003BEC0BF030C182F40401300E82273BEC14
:103020000BF031C182F40401300E82273BEC0BF02F
:1030300004012E0E826F3BEC0BF032C182F40401CE
:10304000300E82273BEC0BF033C182F40401300ECA
:1030500082273BEC0BF004016D0E826F3BEC0BF012
:1030600004012C0E826F3BEC0BF04FC100F150C1FC
:1030700001F151C102F152C103F10101B6EC1FF09F
:1030800079EC1DF00401480E826F3BEC0BF004015B
:103090007A0E826F3BEC0BF004012C0E826F3BEC3E
:1030A0000BF066C100F167C101F168C102F169C1AD
:1030B00003F10101B6EC1FF079EC1DF00401630E81
:1030C000826F3BEC0BF004012C0E826F3BEC0BF09B
:1030D00066C100F167C101F168C102F169C103F184
:1030E00001010A0E046F000E056F000E066F000E40
:1030F000076F29EC1FF0000E046F120E056F000E13
:10310000066F000E076F49EC1FF0B6EC1FF02AC1E6
:1031100082F40401300E82273BEC0BF02BC182F4C9
:103120000401300E82273BEC0BF02CC182F4040129
:10313000300E82273BEC0BF02DC182F40401300EDF
:1031400082273BEC0BF02EC182F40401300E822763
:103150003BEC0BF02FC182F40401300E82273BECD4
:103160000BF030C182F40401300E82273BEC0BF0EF
:1031700004012E0E826F3BEC0BF031C182F404018E
:10318000300E82273BEC0BF032C182F40401300E8A
:1031900082273BEC0BF033C182F40401300E82270E
:1031A0003BEC0BF00401730E826F3BEC0BF004015F
:1031B0002C0E826F3BEC0BF013EC20F059C100F1A8
:1031C0005AC101F184EC1AF00FB2EAEF18F00FA027
:1031D0001CEF19F004012C0E826F3BEC0BF0200E5B
:1031E000F86EF76AF66A04010900F5CF82F43BEC49
:1031F0000BF00900F5CF82F43BEC0BF00900F5CFA2
:1032000082F43BEC0BF00900F5CF82F43BEC0BF0C1
:103210000900F5CF82F43BEC0BF00900F5CF82F406
:103220003BEC0BF00900F5CF82F43BEC0BF009000E
:10323000F5CF82F43BEC0BF045EC0BF00F90109EB9
:1032400012985AEF19F00401630E826F3BEC0BF0F9
:1032500004012C0E826F3BEC0BF060EC19F00401C2
:103260002C0E826F3BEC0BF0D3EC19F004012C0E0A
:10327000826F3BEC0BF04FEC1AF004012C0E826FC6
:103280003BEC0BF00101F80E006FCD0E016F660EE6
:10329000026F030E036F75EC19F004012C0E826FA0
:1032A0003BEC0BF065EC1AF045EC0BF05AEF19F023
:1032B00045EC0BF00301C26B0790109269EF1CF014
:1032C000D8900E0E2FEC09F0E8CF00F10F0E2FEC86
:1032D00009F0E8CF01F1100E2FEC09F0E8CF02F170
:1032E000110E2FEC09F0E8CF03F10101000E046F7D
:1032F000000E056F010E066F000E076F49EC1FF000
:10330000B6EC1FF02AC182F40401300E82273BEC98
:103310000BF02BC182F40401300E82273BEC0BF042
:103320002CC182F40401300E82273BEC0BF02DC13E
:1033300082F40401300E82273BEC0BF02EC182F4A4
:103340000401300E82273BEC0BF02FC182F4040104
:10335000300E82273BEC0BF030C182F40401300EBA
:1033600082273BEC0BF031C182F40401300E82273E
:103370003BEC0BF004012E0E826F3BEC0BF032C1E4
:1033800082F40401300E82273BEC0BF033C182F44F
:103390000401300E82273BEC0BF004016D0E826FAE
:1033A0003BEC0BF01200120E2FEC09F0E8CF00F10D
:1033B000130E2FEC09F0E8CF01F1140E2FEC09F0F9
:1033C000E8CF02F1150E2FEC09F0E8CF03F101016F
:1033D0000A0E046F000E056F000E066F000E076FD9
:1033E00029EC1FF0000E046F120E056F000E066F21
:1033F000000E076F49EC1FF0B6EC1FF02AC182F4F3
:103400000401300E82273BEC0BF02BC182F4040147
:10341000300E82273BEC0BF02CC182F40401300EFD
:1034200082273BEC0BF02DC182F40401300E822781
:103430003BEC0BF02EC182F40401300E82273BECF2
:103440000BF02FC182F40401300E82273BEC0BF00D
:1034500030C182F40401300E82273BEC0BF00401F2
:103460002E0E826F3BEC0BF031C182F40401300E62
:1034700082273BEC0BF032C182F40401300E82272C
:103480003BEC0BF033C182F40401300E82273BEC9D
:103490000BF00401730E826F3BEC0BF012000A0E6E
:1034A0002FEC09F0E8CF00F10B0E2FEC09F0E8CF7C
:1034B00001F10C0E2FEC09F0E8CF02F10D0E2FEC0C
:1034C00009F0E8CF03F184EF1AF0060E2FEC09F0B3
:1034D000E8CF00F1070E2FEC09F0E8CF01F1080E5C
:1034E0002FEC09F0E8CF02F1090E2FEC09F0E8CF3C
:1034F00003F184EF1AF0010113EC20F0078457C1A7
:1035000000F158C101F107940101E80E046F800E2B
:10351000056F000E066F000E076F29EC1FF0000EFE
:10352000046F040E056F000E066F000E076F49EC66
:103530001FF0880E046F130E056F000E066F000E4D
:10354000076F18EC1FF00A0E046F000E056F000ED7
:10355000066F000E076F49EC1FF0B6EC1FF001017B
:103560002967B8EF1AF00401200E826FBBEF1AF042
:1035700004012D0E826F3BEC0BF030C182F404018C
:10358000300E82273BEC0BF031C182F40401300E87
:1035900082273BEC0BF032C182F40401300E82270B
:1035A0003BEC0BF004012E0E826F3BEC0BF033C1B1
:1035B00082F40401300E82273BEC0BF00401430E31
:1035C000826F3BEC0BF0120087C32AF188C32BF10A
:1035D00089C32CF18AC32DF18BC32EF18CC32FF13B
:1035E0008DC330F18EC331F190C332F191C333F109
:1035F0000101296B61EC20F0D8EC1FF00101000EF5
:10360000046F000E056F010E066F000E076F29ECA8
:103610001FF00E0E0C6E00C10BF018EC09F00F0E2F
:103620000C6E01C10BF018EC09F0100E0C6E02C10B
:103630000BF018EC09F0110E0C6E03C10BF018EC36
:1036400009F004017A0E826F3BEC0BF004012C0EA2
:10365000826F3BEC0BF00401350E826F3BEC0BF0FC
:1036600004012C0E826F3BEC0BF060EC19F0F0EFD4
:1036700013F087C32AF188C32BF189C32CF18AC3C5
:103680002DF18BC32EF18CC32FF18DC330F18EC37E
:1036900031F190C332F191C333F10101296B61EC37
:1036A00020F0D8EC1FF0880E046F130E056F000E8B
:1036B000066F000E076F1DEC1FF0000E046F040E66
:1036C000056F000E066F000E076F29EC1FF0010159
:1036D000E80E046F800E056F000E066F000E076F78
:1036E00049EC1FF00A0E0C6E00C10BF018EC09F04B
:1036F0000B0E0C6E01C10BF018EC09F00C0E0C6EE9
:1037000002C10BF018EC09F00D0E0C6E03C10BF0AA
:1037100018EC09F004017A0E826F3BEC0BF0040107
:103720002C0E826F3BEC0BF00401360E826F3BECEB
:103730000BF004012C0E826F3BEC0BF04FEC1AF0F7
:10374000F0EF13F087C32AF188C32BF189C32CF162
:103750008AC32DF18BC32EF18CC32FF18DC330F1B1
:103760008FC331F190C332F191C333F1010161ECA8
:1037700020F0D8EC1FF0000E046F120E056F000E43
:10378000066F000E076F29EC1FF001010A0E046F8F
:10379000000E056F000E066F000E076F49EC1FF05C
:1037A000120E0C6E00C10BF018EC09F0130E0C6E2B
:1037B00001C10BF018EC09F0140E0C6E02C10BF0F5
:1037C00018EC09F0150E0C6E03C10BF018EC09F0A3
:1037D00004017A0E826F3BEC0BF004012C0E826F19
:1037E0003BEC0BF00401370E826F3BEC0BF0040155
:1037F0002C0E826F3BEC0BF0D3EC19F0F0EF13F0D2
:1038000087C32AF188C32BF189C32CF18AC32DF118
:103810008BC32EF18CC32FF18DC330F18EC331F1E8
:1038200090C332F191C333F10101296B61EC20F0B7
:10383000D8EC1FF0880E046F130E056F000E066F94
:10384000000E076F1DEC1FF0000E046F040E056FD5
:10385000000E066F000E076F29EC1FF00101E80E45
:10386000046F800E056F000E066F000E076F49ECA7
:103870001FF0060E0C6E00C10BF018EC09F0070EDD
:103880000C6E01C10BF018EC09F0080E0C6E02C1B1
:103890000BF018EC09F0090E0C6E03C10BF018ECDC
:1038A00009F004017A0E826F3BEC0BF004012C0E40
:1038B000826F3BEC0BF00401380E826F3BEC0BF097
:1038C00004012C0E826F3BEC0BF065EC1AF0F0EF6C
:1038D00013F081B803D02FB027EF1DF007A8E1EF58
:1038E0001CF00101800E006F1A0E016F060E026FB0
:1038F000000E036F4BC104F14CC105F14DC106F13F
:103900004EC107F118EC1FF003BF27EF1DF073EC59
:103910001DF04BC100F14CC101F14DC102F14EC18E
:1039200003F1078225EC1EF018C104F119C105F15D
:103930001AC106F11BC107F1F80E006FCD0E016F21
:10394000660E026F030E036F18EC1FF00E0E0C6E66
:1039500000C10BF018EC09F00F0E0C6E01C10BF05A
:1039600018EC09F0100E0C6E02C10BF018EC09F007
:10397000110E0C6E03C10BF018EC09F00784010165
:1039800013EC20F057C100F158C101F107940A0E61
:103990000C6E00C10BF018EC09F00B0E0C6E01C19F
:1039A0000BF018EC09F00C0E0C6E02C10BF018ECC9
:1039B00009F00D0E0C6E03C10BF018EC09F027EFA7
:1039C0001DF007AA27EF1DF00784010113EC20F07A
:1039D00057C100F158C101F10794060E0C6E00C1E9
:1039E0000BF018EC09F0070E0C6E01C10BF018EC8F
:1039F00009F0080E0C6E02C10BF018EC09F0090E6C
:103A00000C6E03C10BF018EC09F0078462C100F1E1
:103A100063C101F164C102F165C103F10794120EA3
:103A20000C6E00C10BF018EC09F0130E0C6E01C106
:103A30000BF018EC09F0140E0C6E02C10BF018EC30
:103A400009F0150E0C6E03C10BF018EC09F0079885
:103A5000079A0401805181197F0B0DE09EA8FED7C3
:103A600014EE00F081517F0BE126E750812B0F010E
:103A7000AD6E29EF1DF092EF0AF018C100F119C1E7
:103A800001F11AC102F11BC103F1000E046F000E17
:103A9000056F010E066F000E076F49EC1FF029A19C
:103AA00068EF1DF02051D8B468EF1DF018C100F187
:103AB00019C101F11AC102F11BC103F1000E046F1B
:103AC000000E056F0A0E066F000E076F49EC1FF01F
:103AD0001200010104510013055101130651021394
:103AE0000751031312000101186B196B1A6B1B6B42
:103AF00012002AC182F40401300E82273BEC0BF045
:103B00002BC182F40401300E82273BEC0BF02CC158
:103B100082F40401300E82273BEC0BF02DC182F4BD
:103B20000401300E82273BEC0BF02EC182F404011D
:103B3000300E82273BEC0BF02FC182F40401300ED3
:103B400082273BEC0BF030C182F40401300E822757
:103B50003BEC0BF031C182F40401300E82273BECC8
:103B60000BF032C182F40401300E82273BEC0BF0E3
:103B700033C182F40401300E82273BEC0BF01200BB
:103B80002FC182F40401300E82273BEC0BF030C1D0
:103B900082F40401300E82273BEC0BF031C182F439
:103BA0000401300E82273BEC0BF032C182F4040199
:103BB000300E82273BEC0BF033C182F40401300E4F
:103BC00082273BEC0BF01200060E1E6E060E1F6ED7
:103BD000060E206E1E2EEAEF1DF01F2EEAEF1DF0DE
:103BE000202EEAEF1DF08B84020E1E6E020E1F6E59
:103BF000020E206E1E2EFAEF1DF01F2EFAEF1DF0A2
:103C0000202EFAEF1DF08B941200FF0E1F6E1FC0C6
:103C100020F0030E1E6E8B841E2E0BEF1EF0030E83
:103C20001E6E202E0BEF1EF08B941FC020F0030E93
:103C30001E6E1E2E19EF1EF0030E1E6E203E19EF93
:103C40001EF01F2E07EF1EF012000101005305E1C8
:103C5000015303E1025301E1002BE8EC1EF013ECE9
:103C600020F03951006F3A51016F420E046F4B0E34
:103C7000056F000E066F000E076F29EC1FF000C1E4
:103C800004F101C105F102C106F103C107F118C138
:103C900000F119C101F11AC102F11BC103F107B210
:103CA00056EF1EF01DEC1FF058EF1EF018EC1FF041
:103CB00000C118F101C119F102C11AF103C11BF1D0
:103CC000120013EC20F059C100F15AC101F1060EA7
:103CD0002FEC09F0E8CF04F1070E2FEC09F0E8CF44
:103CE00005F1080E2FEC09F0E8CF06F1090E2FECD4
:103CF00009F0E8CF07F118EC1FF000C124F101C171
:103D000025F102C126F103C127F1290E046F000E2F
:103D1000056F000E066F000E076F29EC1FF0EE0E08
:103D2000046F430E056F000E066F000E076F1DEC4B
:103D30001FF024C104F125C105F126C106F127C1F8
:103D400007F129EC1FF000C11CF101C11DF102C1F6
:103D50001EF103C11FF1120E2FEC09F0E8CF04F1A0
:103D6000130E2FEC09F0E8CF05F1140E2FEC09F03B
:103D7000E8CF06F1150E2FEC09F0E8CF07F10D0E94
:103D8000006F000E016F000E026F000E036F29EC32
:103D90001FF0180E046F000E056F000E066F000E68
:103DA000076F49EC1FF01CC104F11DC105F11EC1D4
:103DB00006F11FC107F11DEC1FF06A0E046F2A0EF9
:103DC000056F000E066F000E076F18EC1FF0120053
:103DD000BF0EFA6E200E3A6F396BD890003701375C
:103DE00002370337D8B0F9EF1EF03A2FEEEF1EF08E
:103DF00039073A070353D8B412000331070B80097F
:103E00003F6F03390F0B010F396F80EC5FF0406F8C
:103E1000390580EC5FF0405D405F396B3F33D8B0CF
:103E2000392739333FA90EEF1FF0405139271200CF
:103E3000010138EC20F0D8B012000101035107193C
:103E4000346FFBEC1FF0D8900751031934AF800F8B
:103E500012000101346B1FEC20F0D8A035EC20F0EB
:103E6000D8B012000AEC20F013EC20F01F0E366FD1
:103E70004BEC20F00B35D8B0FBEC1FF0D8A003358D
:103E8000D8B01200362F38EF1FF034B122EC20F0FA
:103E900012000101346B04510511061107110008CD
:103EA000D8A01FEC20F0D8A035EC20F0D8B012003C
:103EB000086B096B0A6B0B6B4BEC20F01F0E366F17
:103EC0004BEC20F007510B5DD8A473EF1FF00651A7
:103ED0000A5DD8A473EF1FF00551095DD8A473EFF4
:103EE0001FF00451085DD8A086EF1FF00451085F51
:103EF0000551D8A0053D095F0651D8A0063D0A5FCF
:103F00000751D8A0073D0B5FD8900081362F60EF96
:103F10001FF034B122EC20F0346B1FEC20F0D8906D
:103F20004FEC20F007510B5DD8A4A3EF1FF0065112
:103F30000A5DD8A4A3EF1FF00551095DD8A4A3EF33
:103F40001FF00451085DD8A0B2EF1FF0003FB2EFA0
:103F50001FF0013FB2EF1FF0023FB2EF1FF0032B43
:103F6000D8B4120034B122EC20F012000101346BFD
:103F70001FEC20F0D8B0120054EC20F0200E366F69
:103F8000003701370237033711EE33F00A0E376F6F
:103F9000E7360A0EE75CD8B0E76EE552372FC8EF78
:103FA0001FF0362FC0EF1FF034B12981D8901200D6
:103FB00001010A0E346F200E366F11EE29F03451D4
:103FC000376F0A0ED890E652D8B0E726E732372F7F
:103FD000E3EF1FF00333023301330033362FDDEFFD
:103FE0001FF0E750FF0FD8A00335D8B0120029B159
:103FF00022EC20F01200045100270551D8B0053DF5
:1040000001270651D8B0063D02270751D8B0073D19
:10401000032712000051086F0151096F02510A6F06
:1040200003510B6F12000101006B016B026B036BFC
:1040300012000101046B056B066B076B1200033560
:10404000D8A012000351800B001F011F021F031F85
:10405000003F32EF20F0013F32EF20F0023F32EF1D
:1040600020F0032B342B032512000735D8A01200B3
:104070000751800B041F051F061F071F043F48EF51
:1040800020F0053F48EF20F0063F48EF20F0072BD7
:10409000342B072512000037013702370337083762
:1040A00009370A370B3712000101296B2A6B2B6B7A
:1040B0002C6B2D6B2E6B2F6B306B316B326B336B2C
:1040C000120001012A510F0B2A6F2B510F0B2B6F7E
:1040D0002C510F0B2C6F2D510F0B2D6F2E510F0BE1
:1040E0002E6F2F510F0B2F6F30510F0B306F31513F
:1040F0000F0B316F32510F0B326F33510F0B336F88
:10410000120000011650FF0A01E11200390EC86EBC
:10411000800EC76E280EC66E000EC56E1550000AC2
:10412000D8B4BCEF20F01550010AD8B4D5EF20F078
:104130001550020AD8B4EEEF20F01550030AD8B497
:1041400007EF21F01550040AD8B42FEF21F01550D5
:10415000050AD8B448EF21F01550060AD8B461EF2B
:1041600021F01550070AD8B47AEF21F01550080A4B
:10417000D8B493EF21F012001650000AD8B4B2EF71
:1041800021F01650010AD8B4B6EF21F01650020AF9
:10419000D8B4BAEF21F01650030AD8B4BEEF21F01C
:1041A0001650040AD8B431EF22F01650000AD8B4E1
:1041B000C6EF21F01650010AD8B4CAEF21F016500C
:1041C000020AD8B4CEEF21F01650030AD8B4D2EFC9
:1041D00021F01650040AD8B431EF22F01650000A2C
:1041E000D8B4D6EF21F01650010AD8B4DAEF21F096
:1041F0001650020AD8B4DEEF21F01650030AD8B4E4
:10420000E2EF21F01650040AD8B431EF22F0165034
:10421000000AD8B4EFEF21F01650010AD8B4F3EF3A
:1042200021F01650020AD8B4F7EF21F01650030A15
:10423000D8B40BEF22F01650040AD8B40FEF22F0D6
:104240001650050AD8B413EF22F01650060AD8B457
:1042500017EF22F01650070AD8B41AEF22F01650C2
:10426000000AD8B41EEF22F01650010AD8B422EF8B
:1042700022F01650020AD8B426EF22F01650030A94
:10428000D8B42AEF22F01650040AD8B42DEF22F049
:104290001650000AD8B435EF22F01650010AD8B4EF
:1042A00039EF22F01650020AD8B43DEF22F0165032
:1042B000030AD8B441EF22F01650040AD8B431EF03
:1042C00022F01650000AD8B44BEF22F01650010A23
:1042D000D8B44FEF22F01650020AD8B453EF22F0B0
:1042E0001650030AD8B457EF22F01650040AD8B477
:1042F00031EF22F01650000AD8B458EF22F01650D1
:10430000010AD8B45CEF22F01650020AD8B460EF6C
:1043100022F01650030AD8B464EF22F01650040AB3
:10432000D8B431EF22F01650000AD8B465EF22F06D
:104330001650010AD8B469EF22F01650020AD8B418
:104340006DEF22F01650030AD8B471EF22F0165028
:10435000040AD8B472EF22F01650050AD8B475EFEB
:1043600022F012009E96C580162A1200E20EC96E37
:10437000162A1200770EC96E162A1200020EE86E77
:104380008AB4E88AE8CFC9FF162A12009E96C58033
:10439000162A1200E20EC96E162A1200790EC96E94
:1043A000162A1200000EC96E162A12009E96C580AB
:1043B000162A1200E20EC96E162A12007A0EC96E73
:1043C000162A120018BC03D0DAC1E8FF04D0185036
:1043D000E844E8441F09E8CFC9FF162A12009E9658
:1043E000C580162A1200E20EC96E162A120011BAF2
:1043F00003D011BC01D003D0050E156E3ED00101D3
:10440000D66707EF22F0100EC96E09EF22F0D6C171
:10441000C9FF162A1200D7C1C9FF162A1200D8C137
:10442000C9FF162A1200D9C1C9FF162A1200C58475
:10443000162A1200FF0E166E1D9E12009E96C58053
:10444000162A1200E20EC96E162A1200760EC96EE6
:10445000162A1200C584162A1200FF0E166E1D9E23
:104460001200C584152A166A12009E96C580162A67
:104470001200E20EC96E162A12007B0EC96E162AB1
:10448000120011AA04D0230EC96E162A12001C0EA7
:10449000C96E162A12009E96C580162A1200E20ED8
:1044A000C96E162A12007C0EC96E162A1200E9D7B0
:1044B0009E96C580162A1200E20EC96E162A1200B8
:1044C0007D0EC96E162A1200DCD79E96C580162A6C
:1044D0001200E20EC96E162A12007E0EC96E162A4E
:1044E0001200CFD7C584162A1200FF0E166E1D9E2D
:1044F00012001650FF0AD8B437EF23F0390EC86EF9
:10450000800EC76E280EC66E000EC56E1550000ACE
:10451000D8B492EF22F01550010AD8B4A6EF22F0D9
:1045200037EF23F01650000AD8B4E4EF22F016500B
:10453000010AD8B4E8EF22F01650020AD8B4F2EF1C
:1045400022F01650030AD8B4F5EF22F01650000AF4
:10455000D8B4FBEF22F01650010AD8B4FFEF22F0D6
:104560001650020AD8B409EF23F01650030AD8B443
:104570000CEF23F01650040AD8B412EF23F01650B3
:10458000050AD8B415EF23F01650060AD8B41BEF6D
:1045900023F01650070AD8B41EEF23F01650080A6D
:1045A000D8B424EF23F01650090AD8B427EF23F02B
:1045B00016500A0AD8B42DEF23F016500B0AD8B4BF
:1045C00030EF23F037EF23F09E96C58036EF23F0CF
:1045D00017B004D04E0EC96E36EF23F0500EC96EE0
:1045E00036EF23F0C58436EF23F0152AFF0E166E42
:1045F000128037EF23F09E96C58036EF23F017B078
:1046000004D04F0EC96E36EF23F0510EC96E36EF4F
:1046100023F0C58636EF23F0C9CF24F0C59AC588AC
:1046200036EF23F0C58636EF23F0C9CF25F0C59AC3
:10463000C58836EF23F0C58636EF23F0C9CF26F0C4
:10464000C59AC58836EF23F0C58636EF23F0C9CF6B
:1046500027F0C58AC58836EF23F0C58436EF23F0EE
:10466000FF0E166E12861D9C37EF23F0162A1200DD
:1046700012B012D012B213D012B414D012A612007B
:1046800007B01200129624C028F025C029F026C0D9
:104690002AF027C02BF01200129012821200129200
:1046A0001284120000011650FF0A04E11294166AE7
:0646B00079EC22F012007B
:10BF0000E844F926000C160C2B0C3F0C520C640C68
:10BF1000760C860C960CA50CB30CC10CCF0CDC0C6B
:06BF2000E80CF40C000C1B
:00000001FF
